:020000020000FC
:100000000C94B20FE2C100000000000000000000EC
:1000100000000000000000000000000000000000E0
:10002000000000002EC000000000000098C000008A
:1000300000000000000000000000000000000000C0
:10004000A1C000000000000000000000000000004F
:100050000000000002030406080C10182030406065
:1000600080000406080C10182030406080A0C000FA
:100070000003070F1F000D0D0403060D0502030208
:1000800002004FB662FD0DC0552049F00994C52D00
:10009000C095089483FDC795C093B20064604FBEBD
:1000A0001895C0910401089483FDC795C093B200D0
:1000B0006B7FC0910401CF3F09F419C04FBE2B984C
:1000C0002C982D9818952B982C982D9876FD0DC06E
:1000D00065FD0BC0C5E0CA95F1F7C0915101C0FDA7
:1000E0002A9AC1FD289AC2FD299A4FBE18952092DE
:1000F000B200CC27C160C7BB6460F7CFC8CF70FF28
:10010000C6CF65FDC4CF2B9AC2CF70FFC0CF65FDAF
:10011000BECF2C9ABCCF70FFBACF65FDB8CF2D9A59
:10012000B6CF2A9870FFB3CF65FDB1CFC1E4CA95B1
:10013000F1F72B9AACCF289870FFA9CF65FDA7CF18
:10014000C1E4CA95F1F72C9AA2CF299870FF9FCFEE
:1001500065FD9DCFC1E4CA95F1F72D9A98CF4FB6B2
:10016000C0916F00CD7FC0936F006E7FC0918400FF
:10017000CE0DD0918500DF1DD0938900C0938800FB
:100180004FBE18953FB68F7EADB3A170A2118061AE
:10019000A0E0ADBBA0916E00AE7FA0936E007894FE
:1001A000A0910801AA2341F085FD2BC0A091080170
:1001B000AA95A093080125C040E050E085FD15C038
:1001C000A9B196FDA095A2FD4FEFA3E096FDA2E098
:1001D000A0936900AA27A160ACBB8D7FA9B196FD51
:1001E000A095A2FD5FEF451739F7A0E461FDA0934C
:1001F000080185FD03C0A0E4A093080140933601E7
:10020000816085FD0EC0A0910901AA2331F0A09163
:100210000901AA95A093090104C08061AA27A160E1
:10022000ACBB80FF0AC0A09136014A2F61FF8E7FD0
:1002300085FD01C000C0409301014091540144304C
:1002400009F004C0A0910101A0930301A52DA034E1
:1002500008F06860A0910001A395A093000161F0EF
:10026000F894A0916E00A160A0936E0084FF02C07C
:10027000A1E0ADBB3FBE1895A0911401A395A0933A
:10028000140142E050910801552329F085FF03C075
:100290005A9550930801A0913601A13018F0209290
:1002A00039010DC020923A0120924301A0913901F9
:1002B000AF5FA093390118F0AFEFA0933901B09070
:1002C000010150915401523049F466FF91F0A2E3CC
:1002D000BA1678F0A0912601A0930101533049F499
:1002E00066FF39F0A2E3BA1620F0A0916001A09356
:1002F0000101509102015B1521F010F05A9501C0E7
:100300005395509302014A95D1F65091430153956C
:1003100009F45A9550934301A0914401AA95A093E2
:10032000440109F046C0A1E0A093440145E0A0913A
:1003300045015A17F0F1A09146015A1728F441E0FF
:10034000A3E0A093440107C0A09147015A1718F4F5
:1003500041E040934401D0903C01C0900301DC1483
:10036000A8F0A0915401A430D9F066FD0FC0C0924E
:100370003C01539511F0A0914501A0934301A1E0E8
:10038000A0934401ACE3A093020113C0A0913C01EF
:10039000A40F20F45FEF50933C0102C0A0933C01F6
:1003A000A0913C01AF3F29F4AFEFA0933A01A09395
:1003B0004301F894A0916E00A160A0936E0084FFA9
:1003C00002C0A1E0ADBB3FBE18953FB6409184008E
:1003D000509185008F7EADB3A170A2118061A0E025
:1003E000ADBBA0916E00AE7FA0936E00789481FDAE
:1003F00025C0A2E096FDA3E0A09369008260A9B1A8
:1004000096FDA095A2FF05C04093050150930601FB
:100410001FC1A3E096FDA2E0A0936900AA27A160F6
:10042000ACBB8D7F85FF01C006C140E0A9B196FD40
:10043000A095A2FD00C140933601EFC0A3E096FD58
:10044000A2E0A09369008D7F61FF72C0A2E096FDDB
:10045000A3E0A0936900AA27A160ACBB826040938F
:10046000310150933201A0902F014A19B090300110
:100470005B09BB24A22C4C38520518F4209235019C
:1004800049C0A0917401AA2359F1483C520528F4AF
:10049000A0E1BA2EAAE0AA2E23C04836A1E05A074E
:1004A00028F4A8E0BA2EAFE0AA2E1AC0403DA2E080
:1004B0005A0728F4A4E0BA2EAEE1AA2E11C0403AA1
:1004C000A5E05A0728F4A2E0BA2EACE3AA2E08C091
:1004D0004839A8E05A0720F4A1E0BA2EA8E7AA2ECE
:1004E000C42EA0913301CA1AD52EA0913401DA0A84
:1004F000DD202AF4AFEFC094D094CA1ADA0A209211
:100500003501A8E0A210A0E0CA14DA0618F4A1E0B0
:10051000A093350140933301509334014091310150
:100520005091320140932F015093300142E075C049
:10053000A09105014A1BA09106015A0B94FD60C0D1
:1005400093FD5EC092FD5AC086FF03C0D52EC42E17
:100550000CC05695479591FD51C05695479590FD15
:100560004DC0D52EC42ED694C79461FD19C0AC2DB4
:10057000AC51AD2DA24008F005C0DD2089F4AC2DB2
:10058000A85C70F4A0910701A395AA2311F0A09391
:100590000701AA3008F44FC02092360181604BC099
:1005A000A0910701AA2319F0AA95A0930701A22CF4
:1005B00050915A0197FD02C0A0906801AAEFAA0EBF
:1005C000A22DA21DCA18DA0A4FB74170442319F0B0
:1005D00040E050E015C0AFEFCA16D20418F04FEF5C
:1005E00050E00EC0A0914C01CA9E412D000C441F4A
:1005F00050E008F012C04FEF50E00FC056954795FD
:1006000094FF07C0552309F04FEFA42FA6954A0F7A
:10061000521D4F3F520508F04FEF40933601816065
:1006200061FF09C0AFE1A095A923AB299A2F8F7D67
:10063000BB2009F48062A0E4A093080185FF03C0F9
:10064000AAE0A093080161FD03C085FD01C08F7E73
:1006500085FD03C0A0E2A0930901F894A0916E006B
:10066000A160A0936E0084FF02C0A1E0ADBB3FBEBD
:10067000189511E00AC013E008C01AE006C01EE198
:1006800004C014E602C018EC00C005E1BB27BA950F
:10069000F1F70A95D9F71A95C1F708952AE338E7D3
:1006A00009C020E33CE806C02AE234EB03C025E29F
:1006B00038EC00C012E0BB272898BA95F1F72C9AC5
:1006C000BA95F1F72C98BA95F1F7289ABA95F1F7FF
:1006D000123009F02B9A123009F42D9AB0914D0185
:1006E000BA95F1F7123009F02B98123009F42D98D1
:1006F000B7E8BA95F1F71A95F1F6022FB22FBA952D
:10070000F1F70A95D9F73A95A9F628980895221B8A
:1007100039E0001F3A9509F40895221F211B18F4AF
:10072000210F8894F6CF0894F4CF622C722CB0E09D
:100730008894B395221F331FE0F737952795889447
:10074000912E802E020B130B10F4192D082D10F48E
:10075000889401C00894661C771CBA9571F7172D10
:10076000062D0895322D11232AF43A9500951095FF
:10077000031B130BF894029F712C002D129F912CD8
:10078000802C7894780C172D921C292DB4E06B2EB8
:100790002695179507956A94D9F7332321F000958C
:1007A0001095031B130B089500915401043009F4B4
:1007B00074C0B0913601B95198F0B72FB67081F47A
:1007C00066FD2BC005E090906601B92DBA9521F029
:1007D0000AE0BA9509F002E1B0911B01B01BE0F00C
:1007E00066FF0AC0B0913E01B0933C01BFEFB093E9
:1007F0004301B1E0B0934401B0910101B093030112
:1008000020921E0120921F0120922001209221019E
:10081000209222016F7B41C0606490906601B92DE7
:10082000BA9579F4B0910201B095BB1FBB1F1B2F85
:10083000B7950B2FB12FB170B3951B2FB02FBE7F83
:1008400025C0B92DBA95BA9581F4B0910201B09541
:10085000BB1FBB1FBB1F1B2FB7950B2FB12FB37037
:10086000B3951B2FB02FBC7F14C0B0910201B0957F
:10087000BB1FBB1FBB1FBB1F1B2FB7950B2FB12F60
:10088000B770B395B3951B2FB02FB87FB0540B2F13
:10089000120900931E0110931F01089510911B016E
:1008A000169500911A010795B0911E01B01B0B2FF0
:1008B000B0911F01B10B1B2F28F40038BFEF1B07AD
:1008C00040F009C00F37120508F405C00FE710E02B
:1008D00002C000E81FEF0093230110932401089544
:1008E00000912301B09120010B0F10912401B091D0
:1008F00021011B1F20E03091240133230AF42A95A3
:10090000B09122012B1F1AF4203F40F00AC02F3073
:1009100008F407C00FEF1FEF2FE003C000E010E066
:1009200020EF30910301B0913B013B1718F43230B6
:1009300030F009C0B0912401BB235AF004C0B0913B
:100940002401BB2332F40093200110932101209352
:10095000220108952091770100912301000F109149
:100960002401111F0E94B20311232AF40038BFEFA3
:100970001B0740F009C00F37120508F405C00FE748
:1009800010E002C000E81FEF002352F0B091020116
:10099000B01B0B2F18F0013008F00AC001E008C0AE
:1009A00000950F5FB09102010B0F08F001C00FEF2F
:1009B0000093250108952091780100912101109163
:1009C00022010E94B20311232AF40130BFEF1B075A
:1009D00040F009C00F3F120508F405C00FEF10E00A
:1009E00002C001E01FEF112352F0B0912501B01BAE
:1009F0000B2F18F0013008F00AC001E008C0009584
:100A00000F5FB09125010B0F08F001C00FEF0093AD
:100A1000030108950FEF677F71FD2AC072FD09C0C1
:100A20006860B0911B01BA3020F0B52DB03408F4E5
:100A3000677FB0917301BB23D9F0B0911B01BB2339
:100A4000B9F00FEF10911B010E948703F894B09149
:100A5000130172FDB5E00B9F112D002D7894112329
:100A600009F00FEFB0913E010B1710F400913E0119
:100A700000933D01089500911A0110911B0100544B
:100A80001140B0913D0110F4BA9501C0B39511F039
:100A9000B0933D0108950E946809B0E074FDB0E094
:100AA000B06CB0937C00B0917A00B068B064B09341
:100AB0007A000E943903B0E074FDB0E0B06CB093EE
:100AC0007C00B0917A00B068B064B0937A00B091C5
:100AD0007A00B6FDFCCF0091780010917900B091BA
:100AE0007A00BF77B0937A000E94BF0927EE209367
:100AF0004801222309F441C030E030934901732EAC
:100B00007694622E6694620E731E262D372D021780
:100B1000130778F080904801B7EEB80DB093480104
:100B200080904901B0E0B81DB0934901260D371DF2
:100B3000EECF80904801909049011091490116959F
:100B40000091480107951695079523E0169507959E
:100B50002A95E1F7209155012A9529F42092480120
:100B6000209249010AC02A9521F0800E911E2A95F3
:100B7000E1F7809248019092490108952091550132
:100B8000B0917A00B6FDFACF00917800109179000B
:100B9000B0917A00BF77B0937A00B0914A01B395D3
:100BA000B0934A01B83060F120924A01B0917201CD
:100BB000BB2321F1112329F0B0914B01BF3F61F01C
:100BC00009C0B0914B010B1739F020F4BB2321F081
:100BD000BA9502C0B395E1F300913B01B0934B018C
:100BE000B03050F400ECB03038F400E8B03020F40D
:100BF00000E4B03008F400E000933B017F7E0895EC
:100C00002130B1F00F3FB3E01B0790F4B7EEBB23E8
:100C100079F0B09148010B17B09149011B0740F4DE
:100C2000B0913B01BB2359F0BA95B0933B0107C08B
:100C3000B0913B01BF3F19F0B395B0933B010091D8
:100C40003B01B0910301B01B10F400910301B0917E
:100C50003C010B1750F000913C01B0913C01BF3FAB
:100C600021F0B0913C01B0933B01502E0093040160
:100C7000B0914A01B73009F47061089502E3F89425
:100C8000B09179010B9F012D000C001F7894B09159
:100C90003B010B1710F000913B0100930101009301
:100CA0000301502E0093040100933E010895209209
:100CB0001A01B0EFB0931B010895F89400918400DD
:100CC0001091850020911401789430911501609065
:100CD00016010093150110931601031B160971FDEF
:100CE00003C077FD7DC027C07090170120931701C6
:100CF0002709222311F00FEF1FEF80901801909029
:100D00001901309318016092190100911501109199
:100D100016010819190920911A0130911B01369505
:100D20002795020F131F10F40FEF1FEF00931A0106
:100D300010931B0129C020911A0130911B01390128
:100D4000B4E08B2EB2E09B2E343010F08A949A944B
:100D5000383010F08A949A94769467948A94E1F7E4
:100D600026193709992021F0169507959A94E1F7ED
:100D7000200F311F20931A0130931B0128F43FEFFD
:100D800030931A0130931B01323008F4706871FF00
:100D900002C0B3E00DC0B0916401009111010238AE
:100DA00038F0B395003A08F0B395B63008F0B5E0E6
:100DB0009B2EB4E08B2E10911B0100911A0124E0B0
:100DC000169507952A95E1F70819120928F0B02F12
:100DD000B250B12FB20910F402E010E0980126C021
:100DE00020911A0130911B01390176946794669421
:100DF000669466942619320906950695200F321DD1
:100E000020931A0130931B01323008F07F7704E001
:100E1000369527953695279526952695201B10F013
:100E2000223008F422E089019090640160FDFECF39
:100E3000E0902B01F0902C016160B0916F00B260E6
:100E4000B0936F00380177FD41C0769467940093AA
:100E50002B0110932C01B92DB330E1F0B0FD04C08B
:100E6000060D171D930106C0000F111F0250120935
:100E700022E030E0B92DB33068F020932D0130939B
:100E80002E0100932701109328016092290170928E
:100E90002A013AC000932D0110932E0120932701BF
:100EA000309328016092290170922A0171FF0DC0D0
:100EB000BFE0B0932D0120922E01B0932901209222
:100EC0002A01B0932B0120922C011EC0669400933E
:100ED0002B01B92DB33091F0B0FD03C0060D262DC6
:100EE00003C0000F025022E0B92DB33038F0209338
:100EF0002D01009327016092290106C000932D0166
:100F0000209327016092290100911C0102FD0350EA
:100F1000013039F495FD0EC0B5E0B06CB0937C00A3
:100F20000DC0023029F4B4E0B06CB0937C0006C070
:100F300095FDF2CFB3E0B06CB0937C00009142011C
:100F4000000F10F4BBE60B270093420160FDFECFBB
:100F5000B2E0B0930E016160B0916F00B260B093E7
:100F60006F00B72FB67001F120911A0130911B016B
:100F7000369527953695279571FF02C0B0E43B0F53
:100F8000F8940091840010918500020F131F1093B4
:100F90008900009388006160B2E0B6BBB0916F0039
:100FA000B260B0936F0078940895606120921D0143
:100FB00020E067FD20E206C0606120921D0120E272
:100FC00067FD20E001E011E077FD11C0B72FB6709A
:100FD00009F06F7E14E100911B01069509F4039559
:100FE0000F3008F00FE071FF02C004E114E160FD72
:100FF00010C0B0911D01BB2361F071FF06C0B0911C
:101000000E01BA95B0930E0111F4706252C00E94A5
:10101000AB07B0917B00BF7BB0937B00B0B7B091C2
:101020007B00B064B0937B00B0911D01B395B09389
:101030001D01B0B777FD06C0B1E071FDB3E0BA9510
:10104000F1F7B0B7B072B21709F028C071FF05C050
:101050000395011708F00A95CACF64FD05C00395F2
:10106000011708F0AFCFC3CF6F7EF89430918400A2
:101070006090850070901A0180901B01370D681CEC
:1010800060928900309388006160B2E0B6BBB09195
:101090006F00B260B0936F00789494CFB0910D015F
:1010A000B13008F48FCF64FD8DCF0A9509F09FCF42
:1010B0007F7D20912D0130912E01F894B2E0B6BBD6
:1010C0000091840010918500020F131F1093890076
:1010D00000938800E0902701F09028016160B091B2
:1010E0006F00B260B0936F007894B72FB67039F08C
:1010F000B0910D0172FFB395B0930D0109C075FF5A
:1011000007C067FD05C064FD03C0BF91BF9188C5DE
:10111000089500E063FF03C064FF01C001E0F8949C
:1011200010911101B7E01B9F212D102D7894200FF5
:1011300026951795269517952695179510931101C5
:10114000183718F4B8E7B093110100911101B0916C
:1011500012010B1720F060622B982C982D9860FDDF
:10116000FECFE0902901F0902A016160B0916F00FC
:10117000B260B0936F000895B2E095FD0AC0F89494
:10118000B0931C0128982A9A62FF01C02D9A789486
:10119000F4C0F894B0931C012898299A62FF01C00A
:1011A0002B9A7894EAC0B3E082FF24C095FD11C069
:1011B00002E0F894B0931C01EBE9F0E000935101D8
:1011C0002D98299862FF02C02C9A01C0289A789421
:1011D000D4C002E0F894B0931C01EBE9F0E0009376
:1011E00051012B982A9862FF02C02C9A01C0289ABC
:1011F0007894C3C095FD0BC0F894B0931C01E5E84A
:10120000F0E02D9862FF01C02C9A7894B6C0F89453
:10121000B0931C01E5E8F0E02B9862FF01C02C9A26
:101220007894ABC0B4E095FD0AC0F894B0931C016B
:101230002A98299A62FF01C02C9A78949EC0F8944B
:10124000B0931C0129982A9A62FF01C02C9A7894C5
:1012500094C0B5E082FF24C095FD11C001E0F89470
:10126000B0931C01E1E9F0E0009351012C9828981B
:1012700062FF02C02B9A01C02A9A78947EC004E0D3
:10128000F894B0931C01E5EAF0E0009351012C982A
:10129000289862FF02C02D9A01C0299A78946DC0E7
:1012A00095FD0BC0F894B0931C01EFE7F0E02C988B
:1012B00062FF01C02B9A789460C0F894B0931C012F
:1012C000EBE8F0E02C9862FF01C02D9A789455C0AD
:1012D000B6E095FD0AC0F894B0931C012998289AAD
:1012E00062FF01C02B9A789448C0F894B0931C0117
:1012F0002A98289A62FF01C02D9A78943EC0B1E0E6
:1013000082FF24C095FD11C004E0F894B0931C0145
:10131000E5EAF0E0009351012B982A9862FF02C0A1
:101320002D9A01C0299A789428C001E0F894B093CE
:101330001C01E1E9F0E0009351012D98299862FF2A
:1013400002C02B9A01C02A9A789417C095FD0BC051
:10135000F894B0931C01EBE8F0E02B9862FF01C019
:101360002D9A78940AC0F894B0931C01EFE7F0E04E
:101370002D9862FF01C02B9A78946F7D08952EE717
:1013800030E0F901209251012B982C982D982A9841
:10139000289829986B7F0895A2E5B1E007E00D93A6
:1013A00007E00D9301E00D9304E00D930FEF0D9313
:1013B0000D930BE00D9302E00D9301E00D9301E01E
:1013C0000D93AEE5B1E001E00D9300E00D9304EB69
:1013D0000D930FEF0D930D930D9303E00D930FEF0E
:1013E0000D9301E00D930FEF0D9305E20D9300EDCA
:1013F0000D9308E70D9308EC0D9304E00D930FEFA8
:101400000D9301E00D9300E00D930AE70D9307E0C3
:101410000D9300E00D9301E00D9300E00D930FEFAD
:101420000D9300E00D930895209159018B7FB091A9
:101430005A019F7DB1FD90629F7BB0915B01B1FD30
:101440009064223011F0886001C0877F08950A956A
:10145000E00FF21DB4910895E4E5F0E0009152012F
:101460000E94270AB0937701E4E5F0E00091530170
:101470000E94270AB0937801E2E6F0E0009158015B
:101480000E94270AB093790100917101002309F4A9
:101490000395013108F001E1B02FB00FB00FB09308
:1014A00045011B2FB10FB10FB00FB0934601B10F23
:1014B000B00FB00FB093470100915801023008F40B
:1014C00002E000931301B0916E010FEFB23009F406
:1014D00000EAB33009F402E800931201E0E7F0E01B
:1014E000009175010E94270AB09340010895089564
:1014F0002091680130916901B0915A01B33009F42B
:101500003E5097FF02C020E03FEFB32FB21B6B2E7F
:10151000B25810F4B2E86B2E00E00395609EB12D36
:10152000BD57D8F300934C01089590680E94780A43
:101530000E943F0320E030E0B0E16B2E0E943B03AD
:10154000B09136012B0F321D6A94C1F7B4E0369585
:101550002795BA95E1F7822E9F770E94780A089521
:10156000F894E3E0F0E0B9E0B7BFB491B078C1F32C
:10157000F894A895B4B7B070B4BFB0916000B861EA
:10158000B0936000B0E0B0936000B4E0BEBFBFEFC6
:10159000BDBF0E94BF09B0E0B5B9BFE3B4B9B0E0C8
:1015A000B8B9B0E0B7B9B0E0BBB9B0E0BAB922247D
:1015B000A0E0B0E02D92AA31E9F7A0E0B1E00FEF92
:1015C0002D920A95E9F7B1E0B09342010E94CC094F
:1015D0000E94580EB0E0B06CB0937C00B0917A00DD
:1015E000B460B068B0937A0000916A0100934D0135
:1015F000B1E0B0930A01F8940E9443030E944E03A5
:101600000E943F030E9451030E943F030E94540323
:101610000E943F030E94F50E0E9443030E94430371
:101620000E944103F8940AEF1AEFA9B196FDA09524
:10163000A2FF1FC01A95C9F70A95B1F7E0E0FCE3D5
:10164000B591B43E39F4B591B03E21F4B591BF3FA8
:1016500009F40CC0E0E0F395F395B591B83F49F477
:10166000B591B43931F4B591BA3A19F4EE27F6953B
:1016700009940E94140A0E942C0A0E94770A0E9470
:10168000780A00916A0100934D010E94BF09B2E0FF
:10169000B5BDB2E0B0938100B2E0B093B100B1E06B
:1016A000B5BBB0936E00B2E0B6BBB0936F00B1E0D3
:1016B000B7BBB0937000B0917B00BF7BB0937B0051
:1016C000B0B7B0917B00B064B0937B000E94390347
:1016D00078940E944B0520921001B3E096FDB2E091
:1016E000B0936900B1E0BDBBBB27B160BCBB8D7FCF
:1016F0000E944303626033E02CE0B0913501BB23CC
:1017000021F42CE03A9509F48DCF0E943F0380FF2D
:1017100089CF8E7FB0913601B23070F3B92FBF718F
:101720000091380100933701B0933801B01721F7C9
:101730002A9519F76D7FB3E096FDB2E0B09369008A
:10174000BB27B160BCBB8D7FB0917401BB2321F47A
:101750008062B92FB0709B2F8F7B209207010E946F
:10176000410385FF05C0B0910701BA3008F08064DD
:101770000E943B0302E085FF01C000E0B09136010A
:10178000B017B0F3F8940E944E030E944E030E94DB
:101790004E0378940E944303209226010E943B034B
:1017A000B0915E01B13008F48AC0B0910A01B13045
:1017B00008F485C085FD1EC0B0913601BF3F08F416
:1017C0007EC0F8940E94570378940E944103B09120
:1017D0003601B130B0F7F8940E944E030E943D03E9
:1017E0000E944E0378940E944103B0913601BF3F9E
:1017F00090F350C3B8E09B2E9068F8940E94780A4A
:1018000078940E944103F8949F770E94780A809010
:101810003601B0913601BF37789408F458C00E9461
:101820003903F8940E94570378949A9429F70E94F8
:10183000950AB82DB550B09369010E944303F894FE
:101840000E948B0E0E94FB0E7894BAE09B2E90684B
:10185000F8940E94780A78940E944103F8949F7744
:101860000E94780A80903601B0913601BF37789493
:1018700060F70E943903F8940E944E030E943D03D2
:101880000E944E0378949A9411F70E94950AB82DFD
:10189000BB5FB09368010E944303F8940E948B0ED3
:1018A0000E94180F78940E944103F8940E94780ACD
:1018B0007894B0913601BF3F08F47CCFEBC2009121
:1018C0003601B09126010B1710F0009326010E94FB
:1018D000410301E0B0915A01B35009F405E0B09121
:1018E0003601B01708F05ACFF8940E9457030E94AF
:1018F00057030E94570378940E94430320920A01E1
:1019000020920B0120920C01B0910B01B395B09382
:101910000B01BF3F91F5B0910C01B395B0930C0151
:10192000B0916C0109E1BA9559F002E3BA9541F022
:101930000DE7BA9529F00AEFBA9511F020920C0143
:10194000B0910C01B017C8F00E94BF090E94390382
:10195000B0910C01BA95B0930C0120920B01B0919B
:101960006B01B0934D01F8940E9457037894B091A5
:101970006A01B0934D010E9441030E943D03B09162
:101980000801BB2319F485FF01C04CCE01E085FDA1
:1019900001C006E0B0913601B01708F4B5CF0E943F
:1019A0004103B0910801BB2309F43CCEF8940E9496
:1019B000BF09209201012092020120920301522CC2
:1019C00020920401209241017894B0915701BB0FFD
:1019D000B0933F0120921E0120921F01209220010E
:1019E000209221012092220120924A0160E070E0C1
:1019F00020921101B8E0B0934A0170610E9439034E
:101A0000B0E074FDB0E0B06CB0937C00B0917A00AF
:101A1000B068B064B0937A00B0917A00B6FDFCCFA4
:101A20000091780010917900B0917A00BF77B0935F
:101A30007A00112309F00FEF00934B010E94BE05BD
:101A4000B8E0B0934A0170610E94140AF894BFEFA5
:101A5000B0933B010E943E06B0910101B0933B015F
:101A6000B0933C01B0933D017894B1E0B093010193
:101A7000B09303015B2EB0930401B0934401B09185
:101A80003A01B0934301B0915A01B33019F49F7DEC
:101A900087FD90627160726020920D010E9468095A
:101AA0000E947F090E9457060E945D060E94570609
:101AB0000E945D060E9457060E94DC070E94D40324
:101AC0000E9489080E94BC080E945D060E94D507FA
:101AD00066FD0E944E0477FF0E940A0577FD0E9472
:101AE0003B050E9489080E94D3080E945D060E945F
:101AF000DC0766FD0E9470040E9489080E9412099A
:101B00000E945D060E94D50766FD0E94AA040E94FD
:101B100089080E9429090E945D060E94DC0766FD73
:101B20000E94DB040E9489080E9468090E945D06E9
:101B30000E94D507B0E074FDB0E0B06CB0937C00BB
:101B4000B0917A00B068B064B0937A000E948908BE
:101B50000E947F090E945D060E94BE0571FF1EC0A3
:101B6000B0913E01B0933B01B0933C01B0913A017A
:101B7000B0934301B1E0B093440118E12CE0B0917F
:101B80000D01B11728F07D7F746020930F0106C00E
:101B9000B0913601B13008F08FCF4CC072FF11C048
:101BA00067FD0FC0B0910F01BA9519F47B7F786083
:101BB00083CFB0930F01B0913601B13008F07CCFE4
:101BC00039C020921001B0913901B13058F0B09174
:101BD0003E01B0933C01B0913A01B0934301B1E0B2
:101BE000B0934401B09139010AEF109176011123AD
:101BF00009F003E0B01708F01DC085FF04C0B091E4
:101C00000801BB23B9F000EF67FF05C0B0913E01AA
:101C1000B0933B0100E2B0911B01B01708F44CCF28
:101C2000B0911001B395B0931001B0913601BB2370
:101C300009F002C020921001F8940E94BF09809020
:101C40005901B2E0B09359010E94140A80925901DF
:101C5000209201012092020120920301522C209235
:101C6000040120923F0160E070E078940E944103FB
:101C70000E94BF0900917601002319F02B9A2C9A3B
:101C80002D9AB0E0B06CB0937C00B0917A00B46053
:101C9000B068B0937A0085FF05C0B0910801BB23FE
:101CA00009F4C0CCB0915F01B13008F061CD28CE0D
:101CB000EDE0F0E00E94840E053A09F01EC0EEE06F
:101CC000F0E00E94840E0A3509F017C03AE0A2E560
:101CD000B1E0E3E0F0E00E94840E0D9331963A9576
:101CE000D1F739E1AEE5B1E0EFE0F0E00E94840E1B
:101CF0000D9331963A95D1F704C00E94CC090E9409
:101D00008B0EE8E2F0E00895F999FECFE1BDF2BD57
:101D1000F89A00B508950E94AE0E3AE0A2E5B1E04F
:101D2000E3E0F0E00D910E94A60E31963A95D1F7CE
:101D300039E1AEE5B1E0EFE0F0E00D910E94A60ED2
:101D400031963A95D1F70E94B90E0895F999FECFD0
:101D500000BDE1BDF2BDFA9AF99A0895EDE0F0E018
:101D60000FEF0E94A60EEEE0F0E00FEF0E94A60E2D
:101D70000895EDE0F0E005EA0E94A60EEEE0F0E046
:101D80000AE50E94A60E089530914E0100914F0180
:101D9000313011F400935201323011F400935301A9
:101DA000333011F400935401343011F40093660180
:101DB000353011F400935501363011F40093580179
:101DC000373011F400936401383011F40093590155
:101DD000393011F400936E013A3011F400935A0136
:101DE0003B3011F400935B01089525E00E9443030A
:101DF0002A95E1F708950E944E030E9451030E9424
:101E000054030E9457030E943D030E944E030E9408
:101E100051030E9454030E9457030E943D030E94F5
:101E20004E030E9451030E9454030E9457030895D9
:101E30000E9457030E9454030E9451030E944E03C4
:101E40000E943D030E9457030E9454030E945103C5
:101E50000E944E030E943D030E9457030E945403B8
:101E60000E9451030E944E03089580904E0190906D
:101E70004F010E944E030E944E030E944E030E9497
:101E80003D038A94B1F70E9457030E943D039A9440
:101E9000D1F70895F8940E94FB0E78940E94F50EF5
:101EA0000E94F50EB1E0B0934E01B1E0B0934F0146
:101EB00020925001F8940E94350F7894B5E06B2E73
:101EC000709036010E944303B09136017B16C1F732
:101ED000B13018F0BF3F70F10CC00E94C40EF894EE
:101EE0000E948B0E0E94FB0EB8E0B09360000E942F
:101EF000F50E6A9429F7B0915001B395B093500153
:101F0000B33008F4D7CF0E94F50EB0914F01B395CE
:101F1000B0934F01F894B0914E01BA95E6E7F0E026
:101F2000EB0FF21D049178940395B0914F01B01717
:101F300008F4BECF0E94F50E0E94F50EB0914E013E
:101F4000B395B0934E01B0914E01BC3008F4ADCFC3
:101F50000E94CC09F8940E948B0EB8E0B093600008
:061F60000E94F50EFDCA0F
:00000001FF
